:1000000018308A0000280000FF00030E8301A100C1
:100010000A08A0008A010408A2007708A300780853
:10002000A4007908A5007A08A6007B08A70083131E
:1000300083128B1D1D280B1846280B1E21288B1898
:1000400049288C308400801E27288C1A4C288C303C
:100050008400001C2D280C184F288C308400801C34
:1000600033288C185228220884002308F70024081B
:10007000F8002508F9002608FA002708FB002008E8
:100080008A00210E8300FF0E7F0E09008A110A12DA
:10009000382A8A110A128B298A110A128D2A8A118A
:1000A0000A12B62A8A110A12A52A0A108A100A11FF
:1000B000820728340C34013406340A108A100A11DD
:1000C0008207203400340A108A100A118207413452
:1000D0005A3400340A108A100A1182072034453439
:1000E0004C3400340A108A100A11820752346534E5
:1000F000713400340A108A100A11820750346F34A8
:10010000733400340A108A100A11820754344834B8
:1001100045344E342034503455345334483420342C
:1001200027345034413452344B34273400340A10CD
:100130008A100A118207523445344634203441343F
:100140005A3449344D3455345434203400340A1070
:100150008A100A1182072034533445345434203431
:1001600041345A3449344D345534543420345434A1
:100170004F34203400340A108A100A118207533495
:1001800045345434203445344C34453456342E34BC
:10019000203454344F3420345A34453452344F349C
:1001A00020342034203400340A108A100A118207C7
:1001B0002034203443344F344E34463449344734A9
:1001C000203445344C344534563441345434493465
:1001D0004F344E342034203400340A108A100A116F
:1001E000F43E03188A0A820050347534733468343C
:1001F000203427345034413452344B3427342034A3
:100200007734683465346E3420344F346B342034A2
:1002100000340A148A100A11820745344C34203401
:1002200054344F3400340A148A100A1182072034DF
:10023000203449344D345034203400340A148A10A8
:100240000A118207503400340A148A100A118207F6
:1002500020345034413452344B3420344D344534FE
:100260004D344F34523449345334453420342034DF
:10027000203400340A148A100A1182075A340034D8
:100280000A148A100A11820720344C34453443344E
:100290005434553452344534203454344134423487
:1002A0004C344534203453344934543445342034A8
:1002B00000340A148A100A11820745344C34003481
:1002C0000A148A100A118207203449344D345034FC
:1002D000203400340A148A100A1182074D34003485
:1002E0000A148A100A1182070C3400340A148A1086
:1002F0000A118207463431345434453420345234A0
:100300004F3454344F34523400340A148A100A11D2
:1003100082072A34003483160510831205108316D1
:10032000851083128510831685118312851183161B
:100330000511831205110B138B138B1B9C29103095
:10034000F700F70BA129000030080317C000C10116
:100350008E0104308D0040088C0083168C130C1520
:10036000831203130B08F7008B1383160317553002
:100370008D00AA308D008C148C18BC290C117708C4
:10038000831203138B041030F700F70BC52900000C
:1003900003178E0105308D0003132F0803178C00FF
:1003A00083168C130C15831203130B08F7008B13A1
:1003B0008316031755308D00AA308D008C148C18CD
:1003C000DF290C117708831203138B041030F70018
:1003D000F70BE829000032080317C000C1018E01A5
:1003E00002308D0040088C0083168C130C1583128C
:1003F00003130B08F7008B138316031755308D007A
:10040000AA308D008C148C18032A0C1177088312E3
:1004100003138B041030F700F70B0C2A00000317AE
:100420008E0103308D000313310803178C008316EF
:100430008C130C15831203130B08F7008B13831610
:10044000031755308D00AA308D008C148C18262A85
:100450000C117708831203138B041030F700F70B8D
:100460002F2A0000630063008B108A110A123328C0
:100470000608303975060317C20003130608F50095
:100480000317C21E532A0313410B4C2A0130AF023B
:100490000030031C0130B002420B522A0130AF077A
:1004A0000318B00A0317421E652A0313400B5E2A85
:1004B0000130B1020030031C0130B2023F0B642A4C
:1004C0000130B1070318B20A0317C401C30144087D
:1004D000273C031C7A2A031D712A43080F3C031C86
:1004E0007A2A43080319C403C3030230C30703185D
:1004F000C40A672A03130B108A110A1233288C1EB0
:100500007F2A1808A8001A08F800A81C892A1812BF
:10051000181600008A110A128E2A7F2A78080317FB
:10052000C60046081F3C031C992A46080D3C031DC3
:10053000A02A7208F20AA03E8400831346088000B5
:1005400003138C128A110A1233287D08033C031C02
:10055000B22A031DAF2A7C08F13C031CB22AFC0A14
:100560000319FD0A8C108A110A123328C30A0C10D1
:100570008A110A12332818308400831700080319DF
:10058000CE2A0630F800F701F70BC42AF80BC32A6D
:100590007B30F700F70BCA2A800BC12A00340317FF
:1005A0001F0EF039F7000F30031308057704880099
:1005B000000008140330F700F70BDC2A08100034A1
:1005C0008810F03083168800831208150000081484
:1005D00000000808080E0F3903179F0003130810C6
:1005E00000000814000000000000000000000808DF
:1005F000080E0F3903179E000313081000308316EE
:100600008800831203171F0EF700F030F7057708F4
:100610001E04F80078089E009E1F102B0313E12A89
:100620009C08031D172B03138810192B03170313A2
:100630008814000008110000081003171D0E9E000A
:100640000F309E051E089F000313CF2203171D08BD
:100650000F399E009F000313CF2200340030831611
:10066000880083128810081108100F3003179800B3
:100670000313BB2201308316E0006008033C031C17
:100680004F2B0330831203179F000313CF22053033
:10069000031798000313BB228316E00A3D2B023098
:1006A000831203179F000313CF228316E001600813
:1006B000033C031C6E2B6008831255208316E10057
:1006C000831203179C018316031361088312031717
:1006D0009D000313E0228316E00A572B83128A152C
:1006E0000A16FD280317190B762B792B40309A0038
:1006F0007A2B9A01013018029A071A0880389B0059
:100700009C011B089D000313E02200340317170807
:10071000F7000C30770203130319972B0A30770286
:100720000319A32B083077020319AB2BB22B031745
:100730009C0101309D000313E02202300317980052
:100740000313BB22BA2B0130031798000230990023
:1007500003137223BA2B03179C0110309D0003135F
:10076000E022BA2B013003179C0017089D000313E9
:10077000E022BA2B00340B138B138B1BBC2B0317FB
:100780003A08BB00BC018E0138088D003A088C0085
:1007900083168C130C15831203130B08F7008B13AD
:1007A0008316031755308D00AA308D008C148C18D9
:1007B000D72B0C117708831203138B040130031716
:1007C0003807BB008E013B088D0039088C0083166A
:1007D0008C130C15831203130B08F7008B1383166D
:1007E000031755308D00AA308D008C148C18F62B11
:1007F0000C117708831203138B04C0308B04003470
:100800006430031790009101A13092009301E13010
:1008100094009501233096000130970064309800D1
:1008200001309900A4309A0001309B00E3309C0015
:1008300001309D0021309E0002309F005E30A000FC
:100840000230A1009A30A2000230A300D530A400EB
:100850000230A5000F30A6000330A7004330A800E7
:100860000330A9007530AA000330AB00A030AC0003
:100870000330AD00C930AE000330AF00EF30B00040
:100880000330B1000D30B2000430B3001530B400B5
:100890000430B5008E0106308D0083168C130C14C5
:1008A00083120C08373C031D562CA02C14308316E1
:1008B0000313E000E1016108133C031C822C0310C8
:1008C000610D103E84008317840A0008E30084034E
:1008D0000008E200600883120317B80083160313B0
:1008E000630883120317BA00831603136208831286
:1008F0000317B9000313BB2302308316E00701304E
:10090000E1075B2C831203178E0106308D00373010
:100910008C0083168C130C15831203130B08F7003D
:100920008B138316031755308D00AA308D008C145D
:100930008C18982C0C117708831203138B0403175F
:1009400003138A150A161C298316E701E8016608B5
:10095000831203178E00831603136508831203178F
:100960008D0083168C130C1483120C08831603134A
:10097000E801E70005308312031798000313BB2238
:1009800083166708EA00E90101306507EB00660895
:10099000EC000318EC0A6C08831203178E00831610
:1009A00003136B08831203178D0083168C130C142A
:1009B00083120C08831603136904E7006A08E80031
:1009C0006708F8006808F90083120034F801F9019B
:1009D000F701FA0103171B08031DF12C1A0803196C
:1009E0000B2D10309C000310980D990DF70DFA0D8A
:1009F0001B087A02031DFE2C1A087702031C072D20
:100A00001A08F702031CFA031B08FA020314F80D74
:100A1000F90D9C0BF32C000003130034031711088D
:100A200099001008980003309B00E8309A000313E7
:100A3000E62478088316EF00831203171108990043
:100A4000100898009B0164309A000313E62479088B
:100A50000317960078089500160899001508980065
:100A60009B010A309A000313E624770803179200CB
:100A700011089900100898009B010A309A0003138E
:100A8000E62479080317960078089500160899005F
:100A9000150898009B010A309A000313E624770892
:100AA0000317930011089900100898009B010A3061
:100AB0009A000313E62477080317940083160313A0
:100AC000EF0803196D2D30306F078312031795005F
:100AD0009700031386237E2D831683120317950137
:100AE000150803135D20003803197E2D0317950A9E
:100AF0009700031386230317702D03138316EF0843
:100B0000031D9B2D83120317920803198A2D831648
:100B100003139B2D9501150803135D20003803195D
:100B2000992D0317950A97000313862303178B2D1E
:100B30000313A32D83163030831203171207950079
:100B40009700031386238316EF08031DC62D831217
:100B5000031792080319AF2D83160313C62D9308AC
:100B60000319B52D83160313C62D9501150803131C
:100B70005D2000380319C42D0317950A970003134D
:100B800086230317B62D0313CE2D83163030831220
:100B900003171307950097000313862330300317BC
:100BA000140795009700031386230034143083162E
:100BB000E200E301E4016308123C031C6B2EE60132
:100BC0006208E5008312A42479088316E1007808FE
:100BD000E000013083120317980099000313722379
:100BE0008316E50165088312402100380319022E9F
:100BF0008316E50A831203179700031386238316CF
:100C0000F22D83120130031798000230990003136C
:100C100072238316E50165088312592100380319F0
:100C20001B2E8316E50A83120317970003138623EE
:100C300083160B2E83120317910183160313640886
:100C400083120317900003130E25DF30031797005C
:100C5000031386238316E50165088312602100389B
:100C600003193C2E8316E50A83120317970003131A
:100C7000862383162C2E8312831661088312031792
:100C80009100831603136008831203179000031367
:100C90000E25831609150030831209190130013C15
:100CA000031D582E0130031798000313BB22492E51
:100CB00004308316E500FA308312031798000313FB
:100CC000BB228316E50B5B2E0230E2076308E30AC2
:100CD0000530E407DB2D83128A150A162A29F7014D
:100CE000F8018316640803106518F707F70CF80C71
:100CF000E518F707F70CF80C6519F707F70CF80C6F
:100D0000E519F707F70CF80C651AF707F70CF80C5C
:100D1000E51AF707F70CF80C651BF707F70CF80C4A
:100D2000E51BF707F70CF80C831200341030F700BE
:100D3000FA010317A401A10CA00C031CA52E220884
:100D4000FA070318A40A2308A407A40CFA0CF90C48
:100D5000F80CF70B9B2E03130034690883166A0204
:100D6000031CBF2E031DBA2E831268088316690266
:100D7000031CBF2E5A30F8000030F900AB2FEC01F5
:100D8000EB01EE01ED01EC08031D042F6B08113C93
:100D9000031C042F6A0883124502031CDF2E031D67
:100DA000D92E440883166902031CD82E8312DF2E25
:100DB00083120030F800F9008316AB2F8312031062
:100DC00083166B0DF9006C0DFA007908443E84001F
:100DD00083137A188317840A0008FA008403000832
:100DE000F8006A087A02031C002F031DFB2E780806
:100DF00069020318002F6B080319EC03EB03042F9F
:100E0000EB0A0319EC0AC32EEC08031D0B2F6B0829
:100E1000113C03180F2F6B080319EC03EB0301308F
:100E20006B07831203179200831603136C08831257
:100E3000031793000318930A0310120DF900130D02
:100E4000FA007908443E840083137A188317840AD1
:100E50000008950084030008940003108316031310
:100E60006B0DF9006C0DFA007908443E8400831381
:100E70007A188317840A0008FA0084030008831292
:100E8000031714029600150897007A08031C7A0FBE
:100E9000970217089900160898009B0105309A00E0
:100EA0000313E6247908031791007808900083164D
:100EB00003136C0883120317A100831603136B0836
:100EC00083120317A000A3010530A2000313962686
:100ED0007908031793007808920003108316031310
:100EE0006B0DF9006C0DFA007908443E8400831301
:100EF0007A188317840A0008FA008403000869023C
:100F0000831203179400831603136A0883120317CE
:100F100095007A08031C7A0F9502150899001408A9
:100F2000980011089B0010089A000313E624780823
:100F30000317120783160313ED0083120317130818
:100F400083160313EE000318EE0A7908EE076D0806
:0A0F5000F8006E08F9008312003467
:101000008316E001E10183120B138B138B1B052860
:10101000013003179800023099008A1103137223DC
:101020008A158316E40164088A11831282208A15C6
:101030000038031927288316E40A83120317970040
:101040008A11031386238A1583161328831201300D
:101050000317980099008A11031372238A158316C7
:10106000E40164088A11831297208A150038031955
:1010700045288316E40A8312031797008A11031385
:1010800086238A15831631288312831661088312FA
:10109000031791008316031360088312031790004F
:1010A0008A1103130E258A15831609140030831242
:1010B00009180130013C031D0A29E8308316E200BB
:1010C0000130E3000030831207180130003A031D9D
:1010D000B828003087190130013C031DB828831659
:1010E0006108033C031C7E28031D7A2860080B3C22
:1010F000031C7E280130E0070318E10A620883120E
:10110000031798008A110313BB228A158316E30A7A
:1011100062081E3C031897281430E4006308E500B9
:101120008A1183126F268A1578088316E2020C3022
:10113000831203179800013099008A110313722358
:101140008A1503108316610CE500600CE400650845
:101150008312031791008316031364088312031785
:1011600090008A1103130E258A15831662288312B4
:10117000003087190130003A031D09290030071893
:101180000130013C031D09298316E008031DCB280B
:10119000E1080319D1280130E0020030031C0130BE
:1011A000E10262088312031798008A110313BB221D
:1011B0008A158316E30A62081E3C0318EA281430D5
:1011C000E4006308E5008A1183126F268A15780807
:1011D0008316E2020C308312031798000130990045
:1011E0008A11031372238A1503108316610CE5001C
:1011F000600CE40065088312031791008316031343
:1012000064088312031790008A1103130E258A15B0
:10121000B828542801300317980099008A11031345
:1012200072238A158316E40164088A118312A720A9
:101230008A150038031928298316E40A8312031734
:1012400097008A11031386238A15831614298312A3
:1012500003108316610CE500600CE400650883123E
:101260000317910083160313640883120317900079
:101270008A1103130E258A1504308316E400C83042
:101280008312031798008A110313BB228A15831651
:10129000E40B3F2909140030831209180130013C86
:1012A000031D7E29003087190130003A03195E2999
:1012B000003007180130003A031D73290030071869
:1012C0000130003A031D68298316051183120515A4
:1012D000003087190130003A031D722983168511E9
:1012E0008312851552298316851183128511831661
:1012F00005118312051183164A2983127308831678
:1013000060078312AF00831661088312B0000318D0
:10131000B00A04300317B800031330080317BA00EB
:1013200003132F080317B9008A110313BB238A156F
:1013300004308316E400C8308312031798008A1122
:101340000313BB228A158316E40B9B2901308312F9
:101350000317980099008A11031372238A158316C4
:10136000E40164088A118312BB208A15003803192E
:10137000C5298316E40A8312031797008A11031301
:1013800086238A158316B12983120130031798002A
:10139000023099008A11031372238A158316E4011F
:1013A00064088A11831282208A1500380319E429FF
:1013B0008316E40A8312031797008A110313862306
:1013C0008A158316D02983128316091400308312DC
:1013D00009180130013C031D172A0030871A01301B
:1013E000003A0319F9290030071A0130003A031DA9
:1013F0000E2A0030871A0130003A031D032A831693
:101400008510831285140030071A0130003A031D3D
:101410000D2A8316051083120514ED298316051075
:10142000831205108316851083128510E42902307B
:101430000317B800BA017408B9008A110313BB235B
:101440008A1504308316E400FA30831203179800DB
:101450008A110313BB228A158316E40B242A8A01FE
:10146000831200288A150A163729B2017408B100C0
:1014700001300317980099008A11031372238A150B
:101480008316E30163088A118312D4208A15003879
:101490000319562A8316E30A8312031797008A1149
:1014A000031386238A158316422A831201300317F9
:1014B0009800023099008A11031372238A1583164B
:1014C000E30163088A118312ED208A15003803199D
:1014D000752A8316E30A8312031797008A110313F0
:1014E00086238A158316612A831283160914003015
:1014F000831209180130013C031D822A8316E00182
:101500008312752A04308316E300FA30831203171E
:1015100098008A110313BB228A158316E30B852AD0
:10152000013083120317980099008A110313722364
:101530008A158316E30163088A118312ED208A1548
:1015400000380319AF2A8316E30A831203179700A2
:101550008A11031386238A1583169B2A831214305B
:101560008316E000E201E101E208031D6A2B610835
:101570005A3C031C6A2B09140030831209180130ED
:10158000013C031D442B01300317980002309900E1
:101590008A11031372238A158316E30163088A11E3
:1015A000831209218A1500380319E22A8316E30AF7
:1015B0008312031797008A11031386238A15831653
:1015C000CE2A8312831662088312031791008316B2
:1015D000031361088312031790008A1103130E2569
:1015E0008A150030871A0130003A0319FD2A0030AD
:1015F000071A0130003A031D162B0030871A0130FC
:10160000003A031D092B0130BF0083168510831299
:1016100085140030071A0130003A031D152B0130E4
:10162000C0008316051083120514F12A83160510D5
:10163000831205108316851083128510BF01C00127
:101640008316E30163088A11831213218A15003877
:101650000319362B8316E30A8312031797008A11A6
:10166000031386238A158316222B8312320803174D
:10167000910003133108031790008A1103130E25FC
:101680008A158316BB2A831202308316E300FA30D0
:101690008312031798008A110313BB228A1583163D
:1016A000E30B472B600883120317B80003133208BB
:1016B0000317BA00031331080317B9008A11031383
:1016C000BB238A1502308316E0070530E1070318B3
:1016D000E20AB42A023083120317B8000313320857
:1016E0000317BA00031331080317B9008A11031353
:1016F000BB238A1503178E0106308D0037308C000E
:1017000083168C130C15831203130B08F7008B132D
:101710008316031755308D00AA308D008C148C1859
:101720008F2B0C117708831203138B04043083165C
:10173000E300FA308312031798008A110313BB22C7
:101740008A158316E30B992B8A01831200288A15C8
:101750000A164329013003179800831603136A08F9
:101760008312031799008A11031372238A158316B3
:10177000EF016F088A11831263208A15003803195C
:10178000CD2B8316EF0A8312031797008A110313D8
:1017900086238A158316B92B831283166E0883124B
:1017A00003179100831603136D088312031790002B
:1017B0008A1103130E258A15DF30031797008A114B
:1017C000031386238A158316EF016F088A1183128B
:1017D0006A208A1500380319F92B8316EF0A831241
:1017E000031797008A11031386238A158316E52BA6
:1017F000831283166C088312031791008316031358
:101800006B088312031790008A1103130E258A15A3
:10181000DF30031797008A11031386238A151230CD
:1018200003179800013099008A11031372238A1557
:101830008316EF016F088A11831272208A1500380F
:1018400003192E2C8316EF0A8312031797008A11AF
:10185000031386238A1583161A2C8312123003175A
:101860009800023099008A11031372238A15831697
:10187000EF016F088A1183127A208A150038031944
:101880004D2C8316EF0A8312031797008A11031356
:1018900086238A158316392C83120034B008031D61
:1018A000552C73082F02031C5E2C73082F02B900FD
:1018B0003008BA000030031C0130BA02B008031D22
:1018C0006D2C73082F0203186D2C2F087302B900BA
:1018D000BA013008031C300FBA028316680883125D
:1018E0003907F8003A08FA000318FA0A7A083602AB
:1018F000031C802C031DAD2C35087802031CAD2C75
:101900000A3035078316E900831236088316EA0089
:101910000318EA0A0A30831239078316EB00831290
:101920003A088316EC000318EC0A68086B02F7000B
:101930006C08FA000030031C0130FA027708F80046
:101940006A087A02031CBB2C0319A82C8312AD2C45
:10195000780869020318BB2C83120130F10083164A
:10196000DF01DE0183123A088316DD008312390895
:101970008316DC00BC2CF101831232088316EA00C6
:10198000831231088316E9008A118312AD268A1565
:101990007908B8007808B7008316680883123707FB
:1019A000F8003808FA000318FA0A7A083402031C0F
:1019B000DF2C031D0C2D33087802031C0C2D0A307C
:1019C00033078316E900831234088316EA000318EC
:1019D000EA0A0A30831237078316EB0083123808AD
:1019E0008316EC000318EC0A68086B02F7006C0819
:1019F000FA000030031C0130FA027708F8006A0888
:101A00007A02031C102D0319072D83120C2D780860
:101A100069020318102D83120130F000122D831675
:101A2000F001831200340908073A003A03192C2EFA
:101A3000831609140030831209180130003A031D7F
:101A4000942D831689140030831289180130013CCB
:101A5000031D942D8316E6010A30E5008A118312D6
:101A6000A4248A157908B4007808B3008316E60127
:101A70000830E5008A118312A4248A157908B6007B
:101A80007808B500B408031D492D33085A3C0318E3
:101A90004B2DB401B3013608023C0318582DFF3A10
:101AA000031D562D35080C3C0318582DB601B50101
:101AB0000310360C8316E1008312350C8316E00008
:101AC0000130EA00831234088316EC0083123308D5
:101AD0008316EB006108EE006008ED008312AA2374
:101AE000103003179800013099008A1103137223F4
:101AF0008A158316E00160088A1183121E218A1557
:101B0000003803198F2D8316E00A831203179700FC
:101B10008A11031386238A1583167B2D831283165D
:101B2000E80183124E242C2E831689140030831270
:101B300089180130003A031DE32D83160914003083
:101B4000831209180130003A031DE32D08300317F2
:101B5000B80003133A080317BA0003133908031730
:101B6000B9008A110313BB238A150A300317B80082
:101B7000031338080317BA00031337080317B90013
:101B80008A110313BB238A150130031798009900AB
:101B90008A11031372238A158316E00160088A11E3
:101BA000831224218A1500380319E22D8316E00AD6
:101BB0008312031797008A11031386238A1583164D
:101BC000CE2D83122C2E831609150030831209198D
:101BD0000130003A031D2C2EB401B301B601B5014A
:101BE0000310360C8316E1008312350C8316E000D7
:101BF0000130EA00831234088316EC0083123308A4
:101C00008316EB006108EE006008ED008312AA2342
:101C1000103003179800013099008A1103137223C2
:101C20008A158316E00160088A1183123A218A1509
:101C300000380319272E8316E00A83120317970032
:101C40008A11031386238A158316132E8312831693
:101C5000E80183124E242C2E8A150A16292A83168F
:101C60006908FA006808840083137A1883178008CB
:101C70000319872E6908ED006808EC006B08EF0077
:101C80006A08EE006F08FA006E08840083137A1861
:101C9000831780080319722E6D08FA006C088400FF
:101CA00083137A1883170008831203179000831692
:101CB00003136F08FA006E08840083137A188317E1
:101CC00000088312031710020319692E83160313E9
:101CD000722E83160313EC0A0319ED0AEE0A031998
:101CE000EF0A422E6F08FA006E08840083137A18F8
:101CF00083178008031D812E6808F8006908F90021
:101D00008A2EE80A0319E90A83122F2E831600305F
:101D1000F800F9008312003403179E019C010A3079
:101D20009D009B019A01180819040319A02E1E0892
:101D30009E0A1807840083131918831700089F0050
:101D40001F082D3C031DB02E01309C001E089E0A6A
:101D50001807840083131918831700089F00BD2EED
:101D60001F082B3C031DBD2E1E089E0A1807840069
:101D700083131918831700089F001F082F3C0318AE
:101D8000742F1F08393C031C742F1F08303C031D9F
:101D9000E92E1E08180784008313191883170008FA
:101DA000783C0319DD2E1E081807840083131918C8
:101DB00083170008583C031DE92E10309D009E0A31
:101DC0001E089E0A18078400831319188317000839
:101DD0009F001D080A3C031D182F1F082F3C0318E5
:101DE000172F1F08393C031C172FA1010A30A00030
:101DF0001B08A3001A08A2008A11031396268A154D
:101E000079080317A1007808A00030301F022007CE
:101E10009A0021089B0003189B0A1E089E0A1807B7
:101E2000840083131918831700089F00ED2E742F68
:101E30001D08103C031D742F1F08603C0318272F3A
:101E40001F087A3C031C272F1F08DF39282F1F0883
:101E50009F002F3C0318302F1F08393C0318382FE0
:101E60001F08403C0318742F1F08463C031C742FA6
:101E70001F082F3C0318552F1F08393C031C552FF2
:101E80001A0DA0001B0DA100A00DA10DA00DA10D0C
:101E9000A00DA10DF030A00530301F0220079A00E0
:101EA00021089B0003189B0A6A2F1A0DA0001B0D26
:101EB000A100A00DA10DA00DA10DA00DA10DF03050
:101EC000A00541301F020A3E20079A0021089B000E
:101ED00003189B0A1E089E0A18078400831319180A
:101EE000831700089F001C2F1D080A3C031D7F2F2D
:101EF0001C0B7F2F9A099B099A0A03199B0A1A083F
:0A1F0000F8001B08F9000313003479
:102000008316EA01EF018312031794010430F800EC
:10201000EB30840083138001840AF80B0B28043012
:10202000F8001030840083178001840AF80B14280C
:1020300083160313E801E901831203179701A03007
:10204000960017089900160898001908FA00180851
:102050008400831319188317800803193328980AFA
:102060000319990A252816081802F7001908FA001A
:102070001708031C170FFA027708F8007A08F9000E
:10208000F908031D4B287808831603136802031808
:10209000E12883120317A030831603136807840016
:1020A000831300082E3C031D5D28EF0101308312CD
:1020B00003179400DD2883160313A03068078400FB
:1020C00083130008203C031D6C28EF0183120317C3
:1020D0009401DD2883160313A0306807840083135E
:1020E00000082F3C03187C28A03068078400831365
:1020F0000008393C0318812883120317DD28831652
:10210000031383120317140B8628DD288316031389
:10211000EF08031D8F28E901EA0A0130EF006A0881
:10212000F70001307702831203199B2802307702EF
:102130000319B928D928EB308316690783120317CE
:10214000950096010318960AA030831603136807BA
:102150008400831300088312031797001508840076
:102160008313161883171708800083160313E90AD0
:10217000DB2810308316690783120317950001309E
:1021800096000318960AA03083160313680784008C
:102190008313000883120317970015088400831324
:1021A000161883171708800083160313E90ADB2823
:1021B00083128316DB288312031783160313E80A9E
:1021C0001C28831203179901EB3098000A128A1514
:1021D00003138C260A168A117908031796007808CB
:1021E0009500961B0E299901EB3098000A128A156A
:1021F00003138C260A168A117908031798007808A9
:102200009700981B11291808003C03181129FF3A60
:10221000031D0E291708683C031811290030F80027
:102220006C2901309900103098000A128A150313A6
:102230008C260A168A1179080317960078089500EB
:10224000961B3A2901309900103098000A128A151D
:1022500003138C260A168A11790803179800780848
:102260009700981B3D299808031D3A2917085A3CE6
:1022700003183D290030F8006C299901EB309800D3
:102280000A128A1503138C260A168A117908031775
:102290009600780895001608A1001508A000A30173
:1022A0000230A2000A12031396260A167808B50017
:1022B0007908B600013003179900103098000A120F
:1022C0008A1503138C260A168A117908B400780837
:1022D000B3000130F800031703138A110A16DA2934
:1022E00001307202A03E8400831300080D3C031DE0
:1022F0001A2A01307202A03E8400831380018316E3
:10230000E801E901E0308400831368088407690864
:102310000A12831263200A168000003803199529D7
:102320008316E90AE80A822983128316E801E90183
:10233000E430840083136808840769080A12831252
:1023400059210A16800000380319AB298316E90ABF
:10235000E80A982983128316E901A030E800EB010E
:10236000E030EA000A128A1583122F260A168A1113
:10237000780879040319CD298316E901A030E80013
:10238000EB01E430EA000A128A1583122F260A169E
:102390008A1178087904031DD929831620084D3C39
:1023A000031DD4298312D9292008573C031D172A5D
:1023B00083120028F8080319162AFD01FC01543085
:1023C000F600103003179800013099000A12031329
:1023D00072230A167608031797000A12031386233E
:1023E0000A160310360C8316E9008312350C831687
:1023F000E8000130EA00831234088316EC008312EF
:1024000033088316EB006908EE006808ED000A1235
:102410008A158312AA230A168A1102308316E8004D
:102420000A128A1583124E240A168A118316F201A3
:10243000A00183128A150A162C2A07083939393A5D
:10244000003A0319962C7D08023C0318962CFF3A9B
:10245000031D2E2A7C08E83C0318962C00308719AF
:102460000130003A03193D2A003007180130003AC4
:10247000031D6D2AF10803196D2A83168510831236
:10248000851083160510831205108316851183129B
:102490008511831605118312051104308316E2009D
:1024A000FA308312031798000A120313BB220A168C
:1024B0008316E20B502A0230F1008312C201C101DF
:1024C00073082F02B5003008B6000030031C01303D
:1024D000B6023608BA003508B9000030871A013054
:1024E000003A03197C2A0030071A0130003A031D14
:1024F000B22AF0080319B22A8316851183128511B6
:102500008316051183120511831685108312851019
:10251000831605108312051004308316E200FA308A
:102520008312031798000A120313BB220A1683169C
:10253000E20B8F2A0230F0008312BF01C001320883
:102540008316EA00831231088316E9000A12831207
:10255000AD260A167908B4007808B3003408B8002C
:102560003308B70003103A0C8316E3008312390CCA
:102570008316E2000230EA00831238088316EC006A
:10258000831237088316EB006308EE006208ED0043
:102590000A128A158312AA230A168A110310360C0E
:1025A0008316E3008312350C8316E2000130EA0043
:1025B000831234088316EC00831233088316EB0071
:1025C0006308EE006208ED000A128A158312AA233E
:1025D0000A168A1183160C148312C30143080B3C9C
:1025E000031C6C2CF4308316E0000130E100003055
:1025F0008312871A0130003A031D552B0030071A49
:102600000130013C031D552BB408031D0F2B33086B
:10261000593C031C0F2B0130B3070318B40A83166F
:1026200060088312031798000A120313BB220A16CC
:1026300083166108E10AE1006008133C0318342B9B
:102640000A30E4006108E5000A1283126F260A16B8
:1026500078088316E4006108E5000A1283126F26E9
:102660000A1678088316E00203108312360C8316CC
:10267000E3008312350C8316E2000130EA00831276
:1026800034088316EC00831233088316EB006308CA
:10269000EE006208ED000A128A158312AA230A16B8
:1026A0008A11C3018316F72A83120030071A0130FA
:1026B000003A031DB12B0030871A0130013C031D85
:1026C000B12BB308031D672BB40803196D2B013020
:1026D000B3020030031C0130B40283166008831279
:1026E000031798000A120313BB220A168316610807
:1026F000E10AE1006008133C0318922B0A30E40061
:102700006108E5000A1283126F260A1678088316FC
:10271000E4006108E5000A1283126F260A167808A1
:102720008316E00203108312360C8316E300831233
:10273000350C8316E2000130EA0083123408831658
:10274000EC00831233088316EB006308EE00620886
:10275000ED000A128A158312AA230A168A11C301F0
:10276000552B003007180130003A031D0F2C0030A4
:1027700087190130013C031D0F2C3608033C031C54
:10278000CB2B031DC72B35080B3C031CCB2B013077
:10279000B5070318B60A831660088312031798005A
:1027A0000A120313BB220A1683166108E10AE1002C
:1027B0006008133C0318F02B0A30E4006108E500C0
:1027C0000A1283126F260A1678088316E40061083D
:1027D000E5000A1283126F260A1678088316E002B3
:1027E00003108312360C8316E3008312350C831614
:1027F000E2000130EA00831234088316EC008312F1
:1028000033088316EB006308EE006208ED000A123D
:102810008A158312AA230A168A11C301B12B00302C
:1028200087190130003A031D6B2C00300718013066
:10283000013C031D6B2CB508031D212CB6080319A0
:10284000272C0130B5020030031C0130B60283167C
:1028500060088312031798000A120313BB220A169A
:1028600083166108E10AE1006008133C03184C2C50
:102870000A30E4006108E5000A1283126F260A1686
:1028800078088316E4006108E5000A1283126F26B7
:102890000A1678088316E00203108312360C83169A
:1028A000E3008312350C8316E2000130EA00831244
:1028B00034088316EC00831233088316EB00630898
:1028C000EE006208ED000A128A158312AA230A1686
:1028D0008A11C3010F2CEE2A83160C1010308312BC
:1028E00003179800013099000A12031372230A1685
:1028F0008316E20162080A1283126A210A1600385E
:1029000003198E2C8316E20A8312031797000A120A
:10291000031386230A1683167A2C83128316E80182
:102920000A128A1583124E240A168A118A150A166B
:102930002F2A831661088312031799008316031345
:1029400060088312031798009B0105309A000A1251
:102950000313E6240A1679088316E3007808E200D8
:10296000630883120317A1008316031362088312FE
:102970000317A000A3010530A2000A120313962634
:102980000A16780883166002E4006108E5007908F9
:10299000031C790FE50201306207EA006308EB00CF
:1029A0000318EB0A03106A0DF9006B0DFA007908A1
:1029B000443E840083137A188317840A0008ED00CC
:1029C00084030008EC000310620DF900630DFA00A7
:1029D0007908443E840083137A188317840A000818
:1029E000FA00840300086C02EE006D08EF007A081C
:1029F000031C7A0FEF026F088312031799008316E6
:102A000003136E088312031798009B0105309A0088
:102A10000A120313E6240A1679088316E9007808D7
:102A2000E8000310620DF900630DFA007908443ED6
:102A3000840083137A188317840A0008EB00840348
:102A40000008EA00650883120317A1008316031328
:102A5000640883120317A000831603136908831206
:102A60000317A30083160313680883120317A20039
:102A70000A12031396260A16780883166A07E600D8
:102A80006B08E7000318E70A7908E7076608F8000B
:0C2A90006708F90083128A150A16C32A91
:10300000840183131F308305063083169F00073029
:1030100083129F00A8018130831699002630980002
:10302000903083129800A901AA010130AB00AC01D5
:10303000AD01AE01AF01B001B101B201B301B40104
:10304000B501B601B701B801B901BA01BB01BC01B4
:10305000BD01BE01BF01C001C101C201C301C40164
:10306000C501C601C701C801C901CA01CB01CC0114
:10307000CD01CE01CF01D001D101D201D301D401C4
:10308000D501D601D701D801D901DA01DB01DC0174
:10309000DD01DE01DF01E001E101E201E301E40124
:1030A000E501E601E701E801E9018316A001A101BC
:1030B000A201A301A401A501A601A701A801A901DC
:1030C000AA01AB01AC01AD01AE01AF01B001B1018C
:1030D000B201B301B401B501B601B701B801B9013C
:1030E000BA01BB01BC01BD01BE01BF01C001C101EC
:1030F000C201C301C401C501C601C701C801C9019C
:10310000CA01CB01CC01CD01CE01CF01D001D1014B
:10311000D201D301D401D501D601D701D801D901FB
:10312000DA01DB018312EA01EB01EC01ED01EE01B2
:10313000EF01F001F101F2016430F300F400F50158
:103140008316DC01DD01DE01DF012030F600FC002A
:103150000330FD0000308500FF308600B930870065
:10316000091489140915851083128510831605101A
:10317000831205108316851183128511831605119C
:1031800083120511071187140730F700F71DD128A6
:10319000073081018130840083130008C0390F3863
:1031A00080006400813084000008C039770480000A
:1031B000B53090007830F80006389200FF30831662
:1031C000920006309F0083121F0838399F00831633
:1031D0000912831294120030940083169400011394
:1031E00083120B168B1583168C160C108C14C030A2
:1031F00083128B040A128A112E2B0A168A15831643
:10320000E00160080A128A11831270210A168A15D9
:103210000038031919298316E00A8312031797004F
:103220000A128A11031386230A168A1583160129A6
:1032300083120A128A11002C0A168A1583160914A1
:103240000030831209180130003A031D2C290A129C
:103250008A11D62D0A168A15831609150030831295
:1032600009190130003A031D38290A1200280A16EC
:10327000831689140030831289180130003A031D27
:1032800044290A12352A0A168316E6010230E5009F
:103290000A128A118312A4240A168A157908B20028
:1032A0007808B1001430EA00EB016B08123C031CF3
:1032B0007D2903106B0D443E8316E000E1010318E5
:1032C000E10AE60183126A088316E5000A128A11F0
:1032D0008312A4240A168A158316600884008313B7
:1032E00061188317840A79088000840378088000B5
:1032F00002308312EA07EB0A552932088316EA00E6
:10330000831231088316E9000A128A118312AD264E
:103310000A168A157908B8007808B7003808B4008A
:103320003708B3008316E6010430E5000A128A115B
:103330008312A4240A168A157908B0007808AF0011
:10334000B008031DA72973082F02031CB0297308B6
:103350002F02B9003008BA000030031C0130BA0255
:10336000B008031DBF2973082F020318BF292F08B7
:103370007302B900BA013008031C300FBA023A08D0
:10338000B6003908B5008316E00160080A128A11F8
:10339000831270210A168A1500380319DD29831655
:1033A000E00A8312031797000A128A110313862377
:1033B0000A168A158316C52983120530031798004B
:1033C000013099000A128A11031372230A168A1512
:1033D0008316E00160080A128A11831276210A1608
:1033E0008A1500380319022A8316E00A831203178C
:1033F00097000A128A11031386230A168A15831668
:10340000EA298312103003179800023099000A123B
:103410008A11031372230A168A158316E0016008C5
:103420000A128A11831285210A168A150038031997
:10343000272A8316E00A8312031797000A128A11BB
:10344000031386230A168A1583160F2A83120A127B
:10345000132D0A168A1170298A158A111D2A8A15B8
:103460003A083602031C552A031D3A2A3508390248
:103470000318552A39083502BD003608BE003A083F
:10348000031C3A0FBE0283165C0883123902BB008C
:103490003A08BC0083165D08031C5D0F502A532AAE
:1034A0008312BC0283166C2A831235083902BD00D0
:1034B0003A08BE003608031C360FBE0239088316D0
:1034C0005C028312BB0083165D088312BC003A08BD
:1034D000031C3A0FBC0283168312BC08031D742A16
:1034E0003B080F3C03187B2ABE08031D7D2A3D08BC
:1034F0000F3C031C7D2A07117E2A0715700B9B2B9E
:10350000103003179800023099000A128A11031331
:1035100072230A168A158316E00160080A128A11BE
:1035200083125D200A168A1500380319A52A83160E
:10353000E00A8312031797000A128A1103138623E5
:103540000A168A1583168D2A831283168C1283120B
:1035500032088316EA00831231088316E9000A1242
:103560008A118312AD260A168A157908B8007808E0
:10357000B70034088316E100831233088316E00095
:103580008A118312992C8A157908ED007808EC00CD
:10359000C0080319082B32086D02031C082B031DF9
:1035A000D52A31086C02031C082B831605108312E0
:1035B000051003103A0C8316E1008312390C8316B0
:1035C000E0000230EA00831238088316EC00831210
:1035D00037088316EB006108EE006008ED000A1260
:1035E0008312AA230A1606308316E000FA308312EB
:1035F000031798000A128A110313BB220A168A15B0
:103600008316E00BF62A0230F0008312C0019B2BD8
:10361000BF080319482B6D083202031C482B031DF9
:10362000152B6C083102031C482B8316851083125E
:10363000851003103A0C8316E1008312390C8316AF
:10364000E0000230EA00831238088316EC0083128F
:1036500037088316EB006108EE006008ED000A12DF
:103660008312AA230A1606308316E000FA3083126A
:10367000031798000A128A110313BB220A168A152F
:103680008316E00B362B0230F0008312BF019B2B18
:103690006D083202031C722B031D522B31086C0281
:1036A0000318722BBF0803196B2B83168510831226
:1036B000851006308316E000FA3083120317980055
:1036C0000A128A110313BB220A168A158316E00B0D
:1036D0005C2B8312BF010130C000831605108312DA
:1036E00005149B2B32086D02031C9B2B031D7C2BA6
:1036F0006C08310203189B2BC0080319952B831605
:1037000005108312051006308316E000FA3083128C
:10371000031798000A128A110313BB220A168A158E
:103720008316E00B862B8312C0010130BF00831685
:10373000851083128514710BBE2C1030031798006E
:10374000023099000A128A11031372230A168A158D
:103750008316E00160080A128A1183125D200A169E
:103760008A1500380319C22B8316E00A8312031747
:1037700097000A128A11031386230A168A158316E4
:10378000AA2B831283168C12730883123507EE005E
:103790003608EF000318EF0AB008031DD32B730897
:1037A0002F02031CDC2B73082F02B9003008BA006B
:1037B0000030031C0130BA02B008031DEB2B730864
:1037C0002F020318EB2B2F087302B900BA0130083F
:1037D000031C300FBA02C20803192B2C6F083002E9
:1037E000031C2B2C031DF82B6E082F02031C2B2C03
:1037F000831605118312051103103A0C8316E1009C
:103800008312390C8316E0000230EA008312380874
:103810008316EC00831237088316EB006108EE0074
:103820006008ED000A128312AA230A1606308316D6
:10383000E000FA308312031798000A128A1103136A
:10384000BB220A168A158316E00B192C0230F100F0
:103850008312C201BE2CC10803196B2C30086F0201
:10386000031C6B2C031D382C2F086E02031C6B2CC1
:10387000831685118312851103103A0C8316E1001B
:103880008312390C8316E0000230EA0083123808F4
:103890008316EC00831237088316EB006108EE00F4
:1038A0006008ED000A128312AA230A160630831656
:1038B000E000FA308312031798000A128A110313EA
:1038C000BB220A168A158316E00B592C0230F10030
:1038D0008312C101BE2C6F083002031C952C031DFE
:1038E000752C2F086E020318952CC20803198E2C14
:1038F000831605118312051106308316E000FA3095
:103900008312031798000A128A110313BB220A16A6
:103910008A158316E00B7F2C8312C2010130C1008F
:103920008316851183128515BE2C30086F02031C87
:10393000BE2C031D9F2C6E082F020318BE2CC1083D
:103940000319B82C8316851183128511063083164E
:10395000E000FA308312031798000A128A11031349
:10396000BB220A168A158316E00BA92C8312C1010B
:103970000130C20083160511831205157108700409
:10398000023C031D092D7008023C031DD82C023097
:103990000317B800031332080317BA0003133108E2
:1039A0000317B9000A128A110313BB230A168A15DA
:1039B0007108023C031DED2C04300317B8000313FB
:1039C00030080317BA0003132F080317B9000A12AF
:1039D0008A110313BB230A168A15F201F101F001C3
:1039E00083168C161030831203179800023099004A
:1039F0000A128A11031372230A168A152A30F60056
:103A00007608031797000A128A11031386230A16F1
:103A10008A1503103A0C8316E1008312390C8316C1
:103A2000E0000230EA00831238088316EC008312AB
:103A300037088316EB006108EE006008ED000A12FB
:0A3A40008312AA230A16272A630046
:02400E00723FFF
:00000001FF
